S01900006F70656E626C745F73746D3332663039312E73726563FF
S3150800000000800020F1050008D5050008D90500087C
S3150800001000000000000000000000000000000000D2
S31508000020000000000000000000000000DD050008D8
S315080000300000000000000000E1050008E5050008D2
S315080000404106000841060008410600084106000866
S315080000504106000841060008410600084106000856
S315080000604106000841060008410600084106000846
S315080000704106000841060008410600084106000836
S315080000804106000841060008410600084106000826
S315080000904106000841060008410600084106000816
S315080000A04106000841060008410600084106000806
S311080000B041060008410600084106000849
S315080000BC10B5064C2378002B07D1054B002B02D024
S315080000CC044800E000BF0123237010BDD0000020B7
S315080000DC00000000A8220008044B10B5002B03D022
S315080000EC0349044800E000BF10BDC04600000000EC
S315080000FCD4000020A8220008002243088B4274D39F
S3150800010C03098B425FD3030A8B4244D3030B8B42FE
S3150800011C28D3030C8B420DD3FF22090212BA030C07
S3150800012C8B4202D31212090265D0030B8B4219D3E8
S3150800013C00E0090AC30B8B4201D3CB03C01A524108
S3150800014C830B8B4201D38B03C01A5241430B8B4250
S3150800015C01D34B03C01A5241030B8B4201D30B0339
S3150800016CC01A5241C30A8B4201D3CB02C01A524160
S3150800017C830A8B4201D38B02C01A5241430A8B4223
S3150800018C01D34B02C01A5241030A8B4201D30B020C
S3150800019CC01A5241CDD2C3098B4201D3CB01C01A26
S315080001AC524183098B4201D38B01C01A5241430930
S315080001BC8B4201D34B01C01A524103098B4201D31E
S315080001CC0B01C01A5241C3088B4201D3CB00C01A8B
S315080001DC524183088B4201D38B00C01A5241430803
S315080001EC8B4201D34B00C01A5241411A00D2014628
S315080001FC524110467047FFE701B5002000F006F89B
S3150800020C02BDC0460029F7D076E770477047C0464E
S3150800021C10B501F03FFE10BD10B501F049FE10BD3A
S3150800022C044B10B51B6900209B0402D500F03AF864
S3150800023C012010BD0008004810B5642000F006F82F
S3150800024C10BDC04610B500F007F810BD014B18805C
S3150800025C7047C046EC00002010B501F0CBFD0E4CE3
S3150800026C236898420FD30D4B1A78002A0CD000221B
S3150800027C1A7090232032DB059A6201F0BBFD084BFD
S3150800028C1B881818206010BD01321A7090231F3273
S3150800029CDB059A61F1E7C046F0000020EE0000206D
S315080002ACEC00002090232022DB059A627047C0469A
S315080002BC0121274A10B513680B43136013681942BA
S315080002CCFCD08022234BD20219680A431A6080227A
S315080002DC196852020A4380211A6089021A680A426E
S315080002ECFCD05A681C491140A42292030A430F21D8
S315080002FC5A60DA6A8A430E390A43DA628022196826
S3150800030C52040A431A608022124992040B6813425B
S3150800031CFCD0F0224B680F4C93434B604B680F4A4A
S3150800032C134003224B604B689343013A13434B60CB
S3150800033C0A3263681340082BFBD1094801F02AF9E5
S3150800034C002000F08BF9236B064A1340236310BD7B
S3150800035C0020024000100240FF7FC2FFFFF8FFFF9B
S3150800036C006CDC02FFFFFCFFF0B5C64600B594B086
S3150800037C00F09AF9FFF79CFF142200210EA801F051
S3150800038C85FF8021454C0903626980260A43626110
S3150800039C6369B6020B4080210393039B6269C90308
S315080003AC0A436261636920250B4080210493049BF0
S315080003BC6369C902334363616369394833400593FA
S315080003CC059B626901270A43626163690B400693C0
S315080003DC069B9023DB0598469D6280230DA99B01FD
S315080003EC0D9300F0B1FE0D9500250DA940460E970C
S315080003FC0F951095119500F0A7FE1C2200210DA84B
S3150800040C01F044FF082200210AA801F03FFFE36926
S3150800041C07A93343E361E369404633400193019BE3
S3150800042C636933436361636903241E400296029B26
S3150800043C02260423099407930C97089600F084FE69
S3150800044C082307A94046079309940C9708960A951A
S3150800045C0B9500F079FEE1235B020D930C23114CEE
S3150800046C0DA9200011930E950F95109512951395BD
S3150800047C01F00EF8A3680C4A1340A36063680B4A94
S3150800048C13402A226360A3689343A36023681F431F
S3150800049C2760FFF7BDFEFFF7BFFEFCE70010024022
S315080004AC0008004800440040FFFBFFFFFFB7FFFFB2
S315080004BC01220A4B82B099691143996199690A40DC
S315080004CC80210092009ADA6949050A43DA61DB69E8
S315080004DC0B400193019B02B07047C04600100240C6
S315080004EC10B5040088B01422002103A801F0CEFE32
S315080004FC134B22689A4201D008B010BD8020114BCC
S3150800050C8004D9690143D9618021DA69C90202409C
S3150800051C0192019A5A690C480A435A615B690B4065
S3150800052C0293029BC0239B0003930223049301337B
S3150800053C069303A90133079300F0A4FCDCE7C04635
S3150800054C00640040001002400004004810B59024D6
S3150800055C00F07CFE2023E405A362134800F07EFD20
S3150800056C124800F07BFD200000F078FD104B114975
S3150800057CDA6911480A40DA61D969104A0140D96129
S3150800058C59691140596159690D4A114059615A699D
S3150800059C0C4902405A61DA690A400121DA619A6902
S315080005AC8A439A6110BDC0460008004800040048FA
S315080005BC00100240FFFFFFFDFFFFFDFFFFFFF7FFE7
S315080005CCFFFFFBFFFFFFFFEF7047C046FEE7C04685
S315080005DC7047C0467047C04610B500F075F810BD98
S315080005EC7047C0460D4885460D480E490E4A0023ED
S315080005FC02E0D458C4500433C4188C42F9D30B4ABD
S3150800060C0B4C002301E013600432A242FBD3FFF724
S3150800061CE7FF01F017FEFFF7A7FEFEE700800020B4
S3150800062CC0000020D000002040250008D000002083
S3150800063C30060020FEE700000121002210B5064B0B
S3150800064C494219611A61D960DA6099629A62FFF7B0
S3150800065C7DFF002010BDC0460010024010B50400F6
S3150800066CFA200E4B80001978FFF746FD0C4B01005B
S3150800067C1868FFF741FD00F0B3FA0123002801D1F1
S3150800068C032C01D9180010BD00222100013800F0F6
S3150800069C7BFA044B1C600023F4E7C046C400002018
S315080006ACC0000020C80000201021064A10B51368A7
S315080006BC00200B431360FFF7D1FFFFF7F9FE00206C
S315080006CC10BDC04600200240034A044B11681B7833
S315080006DC5B1813607047C04608060020C40000204B
S315080006EC70B5041E00D171E02023C35C002B6AD0C0
S315080006FC02212268022513688B43136001F088FBDC
S3150800070C060004E001F084FB801B0A2851D82368F4
S3150800071C5A681542F6D101211A6801250A431A604E
S3150800072C01F076FB060004E001F072FB801B0A2838
S3150800073C3FD823685A681542F6D0227E012A47D03C
S3150800074C80211A688A431A60627E012A59D0402190
S3150800075C1A688A431A60A27E012A4DD020211A688B
S3150800076C8A431A60E27E012A41D010211A680A438C
S3150800077C1A60227F012A35D008211A688A431A6022
S3150800078C627F012A29D004211A688A431A60E16813
S3150800079CA26800200A4321690A4361690A43616811
S315080007AC01390A43DA610023012263622033E254D9
S315080007BC08E08023626A9B021343636205222023A6
S315080007CC0120E25470BDFFF78BFE91E70120F9E793
S315080007DC80211A680A431A60B6E704211A680A4384
S315080007EC1A60D4E708211A680A431A60C8E7102168
S315080007FC1A688A431A60BCE720211A680A431A60E9
S3150800080CB0E740211A680A431A60A4E7202370B59A
S3150800081CC35C013B012B06D98023426ADB021343D6
S3150800082C4362012070BD802403680120A4001A5974
S3150800083C872602431A514A69E23CFF3C1440A04001
S3150800084CC543B6009C592C409C51CC69002C36D01B
S3150800085C012C14D18326B6009C59D20004439C5112
S3150800086C0C688E882404344390269A18B600945142
S3150800087C8C688E89240434439126B60094518124BD
S3150800088C8A69A400002A33D11A592A401A51852498
S3150800089C0A69A400002A33D11A5915401D510A6A4F
S315080008AC012A04D1872189005A58104358508021AF
S315080008BC012089005A5882435A500020B2E7103E4C
S315080008CC9C59D2002C409C51CC688E882404344305
S315080008DC90269A18B60094518C680E8824043443D2
S315080008EC9126B600945181248A69A400002ACBD09B
S315080008FC1A5902431A5185240A69A400002ACBD036
S3150800090C1A5902431A51CAE7202270B5835C0400AF
S3150800091CDBB2012B06D08023426A1B0313434362C6
S3150800092C012070BD02218154016801250A689A4389
S3150800093C0A6001F06DFA060004E001F069FA801B02
S3150800094C0A2806D823685B682B40F6D16362002018
S3150800095CE7E78023626A9B0213436362052220231E
S3150800096C0120E254DDE7C04670B52024045D066814
S3150800097C013CB568012C06D98023426ADB02134375
S3150800098C4362012070BDE0246405254242D0AD01C6
S3150800099CAD0F032D45D00120A84018608B68002B9D
S315080009AC46D10B68C8685B0503432800183000015C
S315080009BC8351C2230C692D0170195B00C450097D43
S315080009CC012903D1C458FF312143C15051791379F8
S315080009DC09021943937975191B041943D3791B0614
S315080009EC0B4329008D31FF310B60517813780902BE
S315080009FC1943937889351B041943D378C0221B06EF
S31508000A0C0B430121FF352B60520083580B4383504F
S31508000A1C0020B7E78023426A9B03134343620120F5
S31508000A2CB0E78023426A1B04134343620120A9E7FB
S31508000A3C4868CC68C0002343B6E7C0462023C25C8E
S31508000A4C0023013A012A06D8036889069B680B40DD
S31508000A5C5B1A581E834118007047C046F0B5CE463F
S31508000A6C4746202480B5045D013C012C09D9802316
S31508000A7C426ADB021343436201200CBC904699463A
S31508000A8CF0BD0468A146002969D02469A40769D079
S31508000A9C4D46D8270C012E197F00BC46F759B84687
S31508000AAC042745462F409760654668D177597F0DD0
S31508000ABC1760D8277F00F559AF3FFF3F2F40DA253F
S31508000ACC6D00D760AC460F2775592F4065461761E0
S31508000ADC775976593F043F0E360C976156614A464C
S31508000AEC1519B935FF352A681A7002681219B93200
S31508000AFCFF321268120A5A7002681219B932FF329A
S31508000B0C1268120C9A7002681219B932FF321268FE
S31508000B1C120EDA7002681219BD32FF3212681A7197
S31508000B2C02681219BD32FF321268120A5A7102682B
S31508000B3C1219BD32FF321268120C9A710268944669
S31508000B4C6444BD34FF342268120EDA710268002937
S31508000B5C0FD1D36820310B43D36000208DE7E468AE
S31508000B6CA40795D18023426A9B0313434362012051
S31508000B7C83E72021136900200B4313617DE777591E
S31508000B8CFF08576095E7C046FF22032330B51400CB
S31508000B9CC5B22B40DB009C4089010A40E4439A40CD
S31508000BAC00280BDB0C4B80089C46C0238000604455
S31508000BBC9B00C1580C402243C25030BD0F23074935
S31508000BCC2B408C46083B9B089B006344D9690C4018
S31508000BDC2243DA61F1E7C04600E100E000ED00E0EF
S31508000BEC0A4A431E012093420ED8C021084A0948D6
S31508000BFC5360036A09061B021B0A0B430362002394
S31508000C0C00209360073313607047C046FFFFFF0050
S31508000C1C10E000E000ED00E00C4B10B5DA6800239C
S31508000C2CD20605D502210A4AD3690B43D361102390
S31508000C3C064AD16804220A4205D001240448134303
S31508000C4CC1692143C161014AD36010BD002002402D
S31508000C5C10060020064B00201A69120606D5054A0E
S31508000C6C5A60054A5A6018690006C00F7047C04694
S31508000C7C0020024023016745AB89EFCD8021034A4A
S31508000C8C002013690B4313617047C04600200240CD
S31508000C9CF8B5050001F0BCF8114C0700012601E077
S31508000CAC6B1C12D1E3681E42FAD12023E268134268
S31508000CBC14D10B4BDA68D20603D4DB6800205B0729
S31508000CCC02D5FFF7A9FF0120F8BD002D04D001F0CD
S31508000CDC9FF8C01BA842E5D90320F5E7E360E8E7CF
S31508000CEC00200240F0B54E465746DE464546E0B56E
S31508000CFC9A4683B02A4B019299461B7E04000E0035
S31508000D0C012B48D001254B4626481D76FFF7C0FF18
S31508000D1C002836D1012C40D0023C63425C410423A6
S31508000D2C6442AC43A0469C46E044002300259B46FF
S31508000D3C18E05346D3404A46594601271A4CD16106
S31508000D4C22699BB23A43226116483380FFF7A0FF0B
S31508000D5C2369BB432361002813D10135EBB2023654
S31508000D6C98450ED920222B0152429A18E1D52022F9
S31508000D7C5146D21A91400A000199D9400B001343E7
S31508000D8CD9E700234A46137603B03CBC90469946ED
S31508000D9CA246AB46F0BD0220F6E701239846C4E707
S31508000DAC1006002050C3000000200240F0B54F4644
S31508000DBC4646D646C0B5304F06003B7E8946012BC3
S31508000DCC57D001233B7603682C48012B34D0FFF708
S31508000DDC5FFF002834D101234A465B421360B3688F
S31508000DEC7568DB025B199D422AD20023244C98466F
S31508000DFC0AE080231B019C46726865449446B368D6
S31508000E0CDB026344AB421CD9022243469246FB6181
S31508000E1C23691A4813432361656123693E321343D8
S31508000E2C2361FFF735FF5246236993432361002854
S31508000E3CDFD04B461D6004E0FFF72AFF002807D0D9
S31508000E4C012000233B761CBC90469946A246F0BD71
S31508000E5C042540220A4CF861236908482B43236170
S31508000E6C236913432361FFF713FF2369AB432361FC
S31508000E7CE7E70220E7E7C0461006002050C300004B
S31508000E8C00200240F0B55746DE464E464546E0B5CC
S31508000E9C0B6885B08A46002B79D0694A00240192E2
S31508000EAC684A9C46914601256346A5402B409846C0
S31508000EBC69D053465A681023170061009F430D3BAF
S31508000ECC8B40DB439B4653469E680097013F8E40FA
S31508000EDC012F63D95B46C5681D402E43C6605B4629
S31508000EEC05682B40032515408D402B430360802352
S31508000EFC5B051A4247D00121019D0F26AB690B43AE
S31508000F0CAB61AB6903250B404F4925408B46AD00B9
S31508000F1CAE400393039BA3089B005B449968B143BB
S31508000F2C9026F605B04212D0484EB04200D17BE06E
S31508000F3C474EB04200D173E0464EB04200D177E03E
S31508000F4C454EB04200D177E00526AE403143996054
S31508000F5C4B4641461B68CD43D10348D449462B40E2
S31508000F6C0B604968930349D44B46294059609968E4
S31508000F7CD3024AD44B4629409960DB6892024BD47B
S31508000F8C2B404A46D36063460134E3408BD105B007
S31508000F9C3CBC90469946A246AB46F0BD5B46876874
S31508000FAC1F405346DB688B401F4301238760476805
S31508000FBCAF4315091D40A5405B463D434560C568D2
S31508000FCC1D40009B2E43C660022B00D087E70726E0
S31508000FDC2640B6000D33B340E508AD0045192F6A17
S31508000FEC9F4353461B69B3401F432F6277E741461D
S31508000FFC0B4349460B6049689303B5D543461943D9
S3150800100C4B4659609968D302B4D5434619434B46A7
S3150800101C9960DB689202B3D542461A431300B0E7CF
S3150800102C0226AE40314392E70126AE4031438EE7A5
S3150800103C0326AE4031438AE70426AE40314386E7A1
S3150800104C0010024000040140000001400004004862
S3150800105C00080048000C00480010004890220300C5
S3150800106CD205904210D02C4A904231D02B4A90424D
S3150800107C16D02B4A904237D02A4A904240D02A4A58
S3150800108C0120934218D070478022284B9202996A05
S3150800109C00200A439A629A6A25490A409A62F2E73C
S315080010AC8022224B1203996A00200A439A629A6A92
S315080010BC20490A409A62E6E780221C4BD203996AB9
S315080010CC00200A439A629A6A1B490A409A62DAE72E
S315080010DC8022164BD202996A00200A439A629A6AAF
S315080010EC16490A409A62CEE78022104B5203996A37
S315080010FC00200A439A629A6A11490A409A62C2E720
S3150800110C80220A4B9203996A00200A439A629A6AC9
S3150800111C0C490A409A62B6E70004004800080048E1
S3150800112C000C00480010004800140048001002404B
S3150800113CFFFFFDFFFFFFF7FFFFFFBFFFFFFFFBFFF3
S3150800114CFFFFEFFFFFFFDFFFF0B54E46DE465746C3
S3150800115C4546E0B50E6883B0002E5CD001239C464C
S3150800116CF34300229A4610E0C368009C2340444689
S3150800117C2343C3600368009C1C40019B5D432543C5
S3150800118C056033000132D34045D063469340334063
S3150800119CF7D01D005D436C006419E44300940C6998
S315080011AC4F686C43A0467C1E0197012CDCD88468DA
S315080011BC009FA3468C686C43A1465C463C40A346FC
S315080011CC4C465F463C435746846044683C40A146BF
S315080011DCCC687443A3464C465F463C434460C4689B
S315080011EC009F3C40A14644464F463C43C460019C84
S315080011FC022CBFD14C69A146FF2B14D82C006C438A
S3150800120CA0464746036A2401E41BA3434C467C4389
S3150800121C23430362AEE7002003B03CBC90469946D4
S3150800122CA246AB46F0BD1B0A5B435B43446AA04629
S3150800123C1C01E41AA34644465F46BC43A0464C46EA
S3150800124C5C43230044462343436293E70121294B1D
S3150800125C82B01A680A431A6001311A681142FCD026
S3150800126CF8211A688A4378390A431A6001225242CD
S3150800127C0192019A20490A400C210192019A5A605E
S3150800128C1C4A53681942FCD113681C490193019BEB
S3150800129C0B4080210193019B89041360154A13683E
S315080012AC0B40FCD11168164801401160536053631A
S315080012BC516B14480140F8205163516B81437838BF
S315080012CC01435163516B7F3881435163516B033032
S315080012DC81435163FF210904D36213630191019978
S315080012EC0020916093608023516A5B040B43536220
S315080012FC02B07047001002400CF8FFF0FFFFF6FE34
S3150800130CFFFFFBFFFFFFFEFF0C20154B70B55A685D
S3150800131C1040082809D00C3843425841114B40421A
S3150800132C1840114B9C46604470BDC0225868520246
S3150800133C10400E4A0F249446604442425041094AD2
S3150800134C40421040084AD96A94462140604401310B
S3150800135C5D68FEF7D1FEAD0C2C4002346043E3E722
S3150800136C00100240005A620200127A000080FEFF4A
S3150800137C10B50400FFF7C8FF084A206053680849EF
S3150800138C1B061B0FCB5CD84060605368054A5B058F
S3150800139C5B0FD35CD840A06010BDC046001002405D
S315080013ACC0220008D022000810B5031E18D103204D
S315080013BC2C4C236B1840022849D0032826D0012828
S315080013CC21D0FFF7A1FF626827491206120F8A5C23
S315080013DC6368D0405B05254A5B0FD35CD84010BDCB
S315080013EC10281FD1C0221F4C9202236B1A4080234F
S315080013FC5B0513431E4A93422FD01E4A934205D0CF
S3150800140C1D4A9342DDD1FFF77FFFE8E702202368E8
S3150800141C184043425841194B40421840184B9C46B9
S3150800142C6044DCE70020122BD9D1C0220D4C1203E4
S3150800143C236B1A4090235B051343124A93420CD034
S3150800144C114A9342E2D0114A9342BAD1DBE7236A96
S3150800145C1840431E9841C003C1E7206A8007C00F95
S3150800146CC003BCE700100240C0220008D0220008C6
S3150800147C00000210000003100000011000EE85FFAA
S3150800148C00127A000000081200000C120000041268
S3150800149C30B5036885B004000D00DB072FD44B6804
S315080014ACC96802680B4329690B43A9690B432D4983
S315080014BC0A401343036043682B4A1340AA68134334
S315080014CC43608368294A13406A6913438360284B2F
S315080014DC984217D0274B98422FD0274B984230D09A
S315080014EC264B984224D0264B984221D0254B98421D
S315080014FC1ED0254B98421BD0244B984218D001205D
S3150800150C05B030BD0020FFF74FFF0028F7D029683B
S3150800151C0029F4D08022AD694B081202954214D0EA
S3150800152CC018FEF7E9FD0004000CE0600020E7E7B0
S3150800153C01A8FFF71DFF0398E7E71020FFF734FF14
S3150800154CE3E71220FFF730FFDFE74000C018FEF78D
S3150800155CD3FD0F4B03400007400F1843E0600020F3
S3150800156CCEE7C046F369FFEFFFCFFFFFFFFCFFFF97
S3150800157C003801400044004000480040004C004040
S3150800158C005000400014014000180140001C0140A6
S3150800159CF0FF0000014B18607047C046C0000020E1
S315080015AC72B6704762B67047F0B5D6464F46464691
S315080015BCC0B58CB002A8FFF7DBFEFA21049B8900A4
S315080015CC18000193FEF798FD00232F4F98462F4BD2
S315080015DCBC1C81462437022505269A4602E0267845
S315080015EC65780234721901325101891A89008918F1
S315080015FC89004846FEF706FE002905D183B29846AF
S3150800160C013B9BB2534539D9A742E8D1AF212048B3
S3150800161C00F00CFC1F4D204E204C214B002723605C
S3150800162C01239946E376434620006360277667765E
S3150800163CA77627776777A760E76026616561FFF766
S3150800164C4FF84B460993174B02A90293164B2000E9
S3150800165C0493042305934B460A930D330B93079770
S3150800166C089703970697FFF7D1F82000FFF74CF970
S3150800167C0CB01CBC90469946A246F0BD013E013DF5
S3150800168C36042D05C8E7C04614230008FF030000DE
S3150800169CD82200080000F0FF0000FFFFF40000202D
S315080016AC00640040E0CC0000E0FF000030B5124BAF
S315080016BC89B002930023114C0200049305930691FA
S315080016CC01AB02A92000FFF74FF9002801D009B099
S315080016DC30BD00F08FFB3230050005E000F064FCED
S315080016EC00F088FBA842F2D801992000FFF7A6F96A
S315080016FC0028F3D1EBE7C046E1070000F400002010
S3150800170C10B58AB003000C0003AA00210A48FFF79B
S3150800171CA5F90023002803D1084A0399914202D05F
S3150800172C18000AB010BD059A0192002AF8D1079B39
S3150800173C23700123F4E7C046F40000206706000076
S3150800174C10B5FFF72DFF10BD70B582B000F078FA12
S3150800175C002801D102B070BDFEF762FD0028F9D051
S3150800176C00F0E8FBFEF768FF00F02EFB0123114A98
S3150800177C80259169AD0519439161926913400193CE
S3150800178C019B00F061FA06002D1AC0360378441C3A
S3150800179C435500F009FC2000B442F7D10321064A50
S315080017AC13680B43136000F04FFA4468FFF7FAFE10
S315080017BCA047CFE7001002400000014070B5541E48
S315080017CCA4B2002A0AD064180134461A0B784D1CA8
S315080017DC8B5500F0E9FB2900A542F7D170BDC04630
S315080017ECF8B507000D4D00260D4C02E0AC68013625
S315080017FC0C3500F0D9FBBC4204D82B689C466444D3
S3150800180CBC4203D8112EF1D1FF20F8BD73009E19E6
S3150800181C044BB6009E19307AF7E7C0463C230008FD
S3150800182C0028000838230008F8B5CE46474680B588
S3150800183C07000068FFF7D4FF0024FF2820D0FFF725
S3150800184C09FA3B1D984680239B000025994605E01E
S3150800185C23689E4211D104354D4516D03B68EC18C9
S3150800186C43465B191E6800F09FFB320000232100DB
S3150800187C0220FFF737FA0028EAD00024FFF7FEF912
S3150800188C20000CBC90469946F8BD0124F6E7C046E4
S3150800189C70B50F4C06000D00A04214D00D4B9942A2
S315080018AC0BD123689D4206D02000802220C09200CE
S315080018BC2900FFF783FF200070BDFFF7B5FF00284E
S315080018CC03D03400EDE7044CEBE70024F3E7C046FD
S315080018DC20030020002800081C010020F0B54F4604
S315080018EC4646D646C0B51E004B0A5B0299460368A7
S315080018FC07000C0015005A1C39D099452DD1043413
S3150800190CE41A3B1D98461F4B3C199A4601339C46D4
S3150800191CE14406E02B78013E237001350134002E94
S3150800192C15D000F041FB4346E31A5345F2D938006B
S3150800193C4946FFF7ADFF071E17D0031D1C00984636
S3150800194C2B78013E237001350134002EE9D1012094
S3150800195C1CBC90469946A246F0BD38004946FFF78E
S3150800196C97FF071E01D00368C9E70020F0E70300BC
S3150800197C4A4604C38022180092004946FFF71EFF08
S3150800198C3B68BAE7FF0100000123034A5B42136078
S3150800199C024A13607047C0461C0100202003002031
S315080019AC134B70B516004A1E04000D001B1A9A42FA
S315080019BC01D9002070BDFFF713FFFF28F9D0601E70
S315080019CC4019FFF70DFFFF28F3D00A4A630A5B029A
S315080019DC934206D02B00320021000748FFF77EFF02
S315080019ECE8E72B00320021000448FFF777FFE1E710
S315080019FCFFFF0308002800081C0100202003002014
S31508001A0CF0B5CE46474680B54C4B4A1E87B0040007
S31508001A1C0D001B1A9A4206D90024200007B00CBCEC
S31508001A2C90469946F0BDFFF7DBFE0600601E40198E
S31508001A3CFFF7D6FE0500FF2EEED0FF28ECD00023CC
S31508001A4C002402938642E8D8042EE6D91628E4D850
S31508001A5C3B4F0533B846994609E00134E4B2122CDB
S31508001A6C62D043461B7899460C239C46E04400F00A
S31508001A7C9BFA4E45F1D163001C19324BA400E3586E
S31508001A8C984605233E009946002406E00134E4B244
S31508001A9C122C4FD033780C36994600F085FA4D4502
S31508001AACF4D163001C19274BA400E3589946052664
S31508001ABC002405E00134E4B2122C39D03E780C37F8
S31508001ACC00F072FAB542F5D163001C191D4BA4003F
S31508001ADC1C19636841464A46551AED1800230393A8
S31508001AEC0123ED0AADB204910593FFF7B3F8002D67
S31508001AFC18D000240AE0802212019446049B013473
S31508001B0C0193A4B263440493A5420BD900F04CFA92
S31508001B1C02A903A8FFF74AF90028ECD00024FFF71E
S31508001B2CADF87AE70124FAE701235B429846A8E761
S31508001B3C0023CFE701235B429946B8E7FFFF03086A
S31508001B4C4C2300083823000800B5104A83B01368E4
S31508001B5C0120013318D0916853688C46D1686344C8
S31508001B6C8C46116963448C46516963448C46916969
S31508001B7C63448C46D26963449B185B4201AA0421D0
S31508001B8C03480193FFF70CFF03B000BD20030020A8
S31508001B9CC02800080D4B18680D4B1B68C0180D4B58
S31508001BAC1B68C0180C4B1B68C0180C4B1B68C0185C
S31508001BBC0B4B1B68C0180B4B1B68C0180A4B1B68D1
S31508001BCCC01843425841C0B27047C04600280008A6
S31508001BDC04280008082800080C2800081028000803
S31508001BEC1428000818280008C02800080A4810B548
S31508001BFC036801330BD109480368013305D0FFF795
S31508001C0C13FE431E9841C0B210BD0120FCE7FFF736
S31508001C1C0BFE0028EFD1F7E7200300201C0100205B
S31508001C2C004870470028000810B5FFF7ADFE10BD38
S31508001C3C10B5FFF7B5FE10BD10B5FFF7E1FE10BDE8
S31508001C4C10B5FFF7A7FF10BD10B5FFF7E9FF10BDDC
S31508001C5C10B5FFF779FF002801D0FFF7C7FF10BDB5
S31508001C6C70B5094C80B2208500F0C4F80A3005001E
S31508001C7C802605E000F098F900F0BCF8A84202D8D6
S31508001C8CE3691E42F6D070BD0044004030B501250C
S31508001C9C0C4C89B023680C22AB432360E1231B024E
S31508001CAC0193002301A9200002930393049306933E
S31508001CBC07930592FFF7ECFB23682B43236009B0C7
S31508001CCC30BDC0460044004070B504000D004029E4
S31508001CDC12D82800ADB2FFF7C3FF002D0BD0013D7B
S31508001CEC631CADB25D1900F05FF920780134FFF77B
S31508001CFCB7FFAC42F7D170BD8421024800F096F8C4
S31508001D0CE7E7C04610240008F8B5204D0E002C78DD
S31508001D1C002C0DD11E4BDA69920606D59B8C1D4AF2
S31508001D2CDBB21370013B3F2B26D900242000F8BDEB
S31508001D3C2024174AD3691C4015D0174C154923780B
S31508001D4C978CCA18577001330A78DBB223709A42FB
S31508001D5CEBD192B20131FFF731FD00232B702378BA
S31508001D6C01243370E2E700F045F80C4B1B6864332A
S31508001D7C9842DAD92C70D8E700F03CF8074B186073
S31508001D8C054B1C7001232B70D0E7C0466505002057
S31508001D9C0044004024050020660500206805002044
S31508001DAC0022064B06491A605A609A60596005214A
S31508001DBC9A601960034B1A607047C04610E000E041
S31508001DCC7FBB00006C0500200022024B1A605A608B
S31508001DDC9A60704710E000E0044B1B68DB0303D5E0
S31508001DEC034A1368013313607047C04610E000E0DD
S31508001DFC6C050020044B1A68044B1868D20301D5ED
S31508001E0C013018607047C04610E000E06C050020F1
S31508001E1C044B1A68044B1868D20301D501301860B4
S31508001E2C7047C04610E000E06C05002010B500F0C5
S31508001E3CBBF8FCE710B500F0ABF8012803D00A4C48
S31508001E4C2378012B00D010BDFFF7D4FF074B084AA7
S31508001E5C1B6812689B18F533FF339842F3D300239B
S31508001E6C2370FFF771FCEEE774050020700500205F
S31508001E7C780500200122054B10B51A70FFF7BAFF3A
S31508001E8C034B1860FFF7D6FF10BDC046740500203B
S31508001E9C7805002010B5FFF753FC00F081F8FFF722
S31508001EAC7FFFFFF7C1FE00F00DF8FFF7E3FF10BD4B
S31508001EBC10B500F079F8FFF78FFF00F013F8FFF76D
S31508001ECCB9FF10BD10B500F073F8FFF76DFB0123D1
S31508001EDC034C2370FFF7DAFE0023237010BDC046AF
S31508001EECCC00002010B582B06B46104CD91D2000D2
S31508001EFCFFF706FC012811D06B462000D91DFFF709
S31508001F0C03FF012801D002B010BD0022084B2000A7
S31508001F1C1A706B46D97900F067F8F4E7044B187019
S31508001F2C6B462000D97900F05FF8E5E77C050020C0
S31508001F3CCC0000207047C04670B50A4D06002B78B9
S31508001F4C0C00012B08D0002B03D1E1B23000FFF7AF
S31508001F5CBBFE00F041F870BDC9B2FFF7A7FB2B78A2
S31508001F6CF1E7C046CC000020054B40201B78013B0E
S31508001F7CDBB2022B02D8034A5B00985A7047C0465C
S31508001F8CCC0000205024000810B5FFF7EDFF10BD5B
S31508001F9C10B500F019F8431E9841C0B210BDC046E2
S31508001FAC10B5FEF749F910BD10B5FEF74BF910BD83
S31508001FBC00224321034B5A5401319A645A521A800F
S31508001FCC9A707047BC050020024B1878431E98413E
S31508001FDCC0B27047BC05002043230021014AD154E6
S31508001FEC7047C046BC050020F8B503780500924C2E
S31508001FFCFF2B0CD02278012A00D0F8BD3733DBB280
S3150800200C352B00D9FCE08D4A9B00D3589F460122FC
S3150800201CE370EF3B2371002322806371FFF7A4FF63
S3150800202CA071FFF7B1FFE071FFF7AEFF012544235E
S3150800203C0822000A20726572A572E252FFF7F4FDB7
S3150800204C4323E35C012B05D04423E15E0029D4DD50
S3150800205C89B207E0FE2302220221E370EE3B2371CC
S3150800206C3433E25243230122E01CE254FFF764FFA7
S3150800207CC3E7FFF779FF6B780138984276DDFF23C3
S3150800208C0122E370BB3BE2526978002900D0C4E018
S3150800209CFFF7DEFD0028D3D1FE230222E370CD3BE9
S315080020AC23711333E2524323E35C012BD2D044232E
S315080020BCE15AD7E74168A06CFFF7BEFD0028EBD0C4
S315080020CCFF230122E370BB3BE252ECE70025FF231A
S315080020DC2571E3706571FFF747FF44230722A0714A
S315080020ECE57125726572E252DDE7FF23E3704768F6
S315080020FCA66C002F00D19DE00025F7193378013620
S3150800210CED18EDB2FFF750FFB742F7D101230022C5
S3150800211CA3800023E571227262722D0EA371083218
S3150800212C4433A572E252BEE7A66CFFF71DFF6A1C84
S3150800213C411E3000FFF77CFD0028ADD0FF23E3706D
S3150800214CFFF712FFA36C01229C4644230138604416
S3150800215CA064E252A7E7FFF7F7FAB1E7002323805A
S3150800216CAEE7FFF701FF6B78834251D3FE230222B9
S3150800217CE370DC3B23712233E25294E7FFF7F4FE5B
S3150800218C6A789042F2D9A16C201DFFF717FBFF2342
S3150800219CA26CE370944644226B786344A3646B7810
S315080021AC0133A3524CE7FF23E37043680122A3646F
S315080021BC4423E25277E7FF23E370214B0721A364FC
S315080021CC0023082223716371A37123726372A372AD
S315080021DC4433E171E25266E7FE23E37000230222E0
S315080021EC23714433E2525EE7FF23E37000236278DF
S315080021FC23716271E380237206224423E25252E76A
S3150800220CFE230222E370DE3B23712433E2524AE7B3
S3150800221C6968201DA1646A78B7E7AA1CA06CFFF749
S3150800222C07FD002800D137E7A26C6B789446634407
S3150800223CA36405E7002569E7BC05002058240008B7
S3150800224C3025000870B500260C4D0D4C641BA410E7
S3150800225CA64209D1002600F021F80A4D0A4C641B47
S3150800226CA410A64205D170BDB300EB5898470136A9
S3150800227CEEE7B300EB5898470136F2E73825000825
S3150800228C38250008382500083C25000803001218D4
S3150800229C934200D1704719700133F9E7F8B5C04677
S315080022ACF8BC08BC9E467047F8B5C046F8BC08BCD6
S309080022BC9E46704775
S315080022C000000000000000000102030406070809D8
S315080022D00000000001020304433A2F576F726B2F68
S315080022E0736F6674776172652F4F70656E424C54D2
S315080022F02F5461726765742F536F757263652F412A
S31508002300524D434D305F53544D333246302F63613F
S315080023106E2E630005020602060307030803090377
S3150800232009040A040B040C040C050D050E050F051B
S315080023300F061006100710080028000800080000FD
S315080023400500000000300008000800000600000034
S3150800235000380008000800000700000000400008D8
S3150800236000080000080000000048000800080000F7
S315080023700900000000500008000800000A000000DC
S3150800238000580008000800000B0000000060000864
S31508002390000800000C0000000068000800080000A3
S315080023A00D00000000700008000800000E00000084
S315080023B000780008000800000F00000000800008F0
S315080023C000800000100000000000010800800000E6
S315080023D011000000008001080080000012000000C3
S315080023E000000208008000001300000000800208B8
S315080023F000800000140000000000030800800000B0
S315080024001500000000800308008000001600000088
S31508002410433A2F576F726B2F736F667477617265C5
S315080024202F4F70656E424C542F5461726765742F36
S31508002430536F757263652F41524D434D305F535448
S315080024404D333246302F72733233322E630000001A
S315080024500800000000000000342100080C220008D3
S315080024600C220008A42000080C2200080C220008F0
S31508002470622100087E200008C0200008D820000835
S315080024800C2200080C2200080C2200080C22000866
S315080024900C2200080C2200080C2200080C22000856
S315080024A00C2200080C2200080C2200080C22000846
S315080024B00C2200080C2200080C2200080C22000836
S315080024C00C2200080C2200080C2200080C22000826
S315080024D00C2200080C2200080C2200080C22000816
S315080024E00C2200080C2200080C2200080C22000806
S315080024F00C2200080C2200080C2200080C220008F6
S31508002500F62000086E21000888210008B22100087C
S315080025100C2200080C2200080C220008C221000820
S315080025200C220008E4210008F421000868210008AC
S30D080025304F70656E424C540021
S30908002538E5000008A4
S3090800253CBD000008C8
S3150800254000127A00010000000400000004000000E8
S705080005F1FC
